:020000040000FA
:0600000060283E300130D3
:08000800A000030EA100831209
:100010008B1C2E288B1031181328B11C2E2864300D
:100020000102031C2D281428152816281728182823
:1000300019281A281B283110B114A810031005190B
:100040000314AA0DA90DA80DB00B2E2831152A08EE
:10005000AF002908AE002808AD00B11081010B11D6
:0A006000210E8300A00E200E0900FF
:1000C000203084008001840A60300402031C62280E
:1000D0001230B000FA228316FF2390008312831699
:1000E0000C3085058701831285018701073099004F
:1000F0000030831691009F008312C8308316810060
:10010000831231309000003083168C00831210303F
:100110008B00BD1B8D28851D7F233D1BBE013D1B14
:10012000BF013D1F682381018E018F010B118B10D0
:100130000B108C130C138C110C108B17AF20311972
:10014000C520CE22B30BAC28031085190314BA0DB9
:10015000F0303A0203190C22BD18A7239E28640030
:10016000311808000B1D08000B11B11031141230AA
:10017000B000051DC0283214831601138312080035
:1001800032108316011783120800321CCC282D0967
:100190000339AD00AE09AF09E4302F02F030031986
:1001A000AF004C302F020C300319AF006C302F021F
:1001B0003C300319AF00EC302F02FC300319AF00C4
:1001C000B3302F02F3300319AF001B302F020F3072
:1001D0000319AF003B302F023F300319AF00BB3093
:1001E0002F02FF300319AF0031110130B7008B131C
:1001F0002030370783169B001C141A088312A400B2
:10020000A50025101030370783169B001C141A0810
:100210008312A3000030370783169B001C141A08B2
:100220008312A2008B1722082D02031D062A230821
:100230002E06FC39031D062A013009303702031D42
:10024000452900302E060339031D2A29BF1F3329F3
:10025000BF13B11703302E060339031D3329BF1B0B
:100260003329BF17B11744302F065439031D3C29D9
:100270003F1F08003F13B11710302F065439031DDC
:1002800045293F1B08003F17B117AF13AF12AF113D
:10029000AF1024082F02031DA72901303702031DC8
:1002A00056293E1856293E14B11710230230370242
:1002B000031D5F29BE185F29BE14B1171223033036
:1002C0003702031D68293E1968293E15B11714230A
:1002D00004303702031D7129BE197129BE15B117EB
:1002E000162305303702031D7A293E1A7A293E1655
:1002F000B117182306303702031D8329BE1A83293C
:10030000BE16B1171A2307303702031D8C293E1B76
:100310008C293E17B1171C2308303702031D95297D
:10032000BE1B9529BE17B1171E2309303702031DC6
:100330009E293F189E293F14B11720230A30370207
:10034000031DA729BF18A729BF14B1172423250807
:100350002F02031D062A01303702031DB4293E1C5B
:10036000B4293E10B117282302303702031DBD29DE
:10037000BE1CBD29BE10B1172A2303303702031D4E
:10038000C6293E1DC6293E11B1172C230430370261
:10039000031DCF29BE1DCF29BE11B1172E23053055
:1003A0003702031DD8293E1ED8293E12B11730232B
:1003B00006303702031DE129BE1EE129BE12B11726
:1003C000322307303702031DEA293E1FEA293E1374
:1003D000B117342308303702031DF329BE1FF32958
:1003E000BE13B117362309303702031DFC293F1C09
:1003F000FC293F10B11738230A303702031D052AA4
:10040000BF1C052ABF10B1173C23062AB70A0B30C0
:10041000370203180800F728B601B3019630B4007C
:100420000130B5000130B70085018701B1139E226C
:10043000AF20B30B562A031085190314BA0DF03000
:100440003A0203198E2AB40B562A013037020319D7
:1004500040230230370203194423033037020319C3
:1004600048230430370203194C230530370203199F
:10047000502306303702031954230730370203197B
:1004800058230830370203195C2309303702031957
:1004900060230A303702031964233708B6080319AA
:1004A000B6000319542AB6039630B400311D182A39
:1004B0003111321C602A2D090339AD00AE09AF0994
:1004C00051302F0655390319752A05302F06553935
:1004D0000319752A15302F0655390319752A553019
:1004E0002F0655390319752A182AAF13AF12AF1109
:1004F000AF108B1320303707BC002F08BB00DC2265
:1005000010303707BC002E08BB00DC220030370754
:10051000BC002D08BB00DC228B17982285018701C7
:10052000B70AB6010B303702031C182A68230800EB
:100530000A30370203190800850187016430B900C9
:1005400033300F1E85000F1A8501FF300F1A870008
:100550000F1E8701AF20311DA02A3111321CB52A90
:100560002D090339AD00AE09AF0951302F065539B9
:1005700003199E2A05302F06553903199E2A153076
:100580002F06553903199E2A55302F065539031960
:100590009E2AB90BA02A850187010800B11F080017
:1005A000B1131030BC003E08BB00DC223030BC0070
:1005B0003F08BB00DC2208003C088B1383169B001D
:1005C0001C141A0883128B173B02031908008B13A3
:1005D0003B0883161C159A003C089B0055309D0073
:1005E000AA309D009C1464009C18F32A1C118312ED
:1005F0008B170800831600309B001C141A08831206
:10060000BD00831610309B001C141A088312BE0014
:10061000831630309B001C141A088312BF00080098
:100620000516080085160800051408008514080042
:10063000871408000715080007140800871608002B
:10064000BD18080007160800BD1808008715080027
:100650000512080085120800051008008510080022
:10066000871008000711080007100800871208000B
:10067000BD18080007120800BD18080087110800FF
:100680000508103A850008000508203A8500080092
:100690000508013A850008000508023A85000800AF
:1006A0000708023A870008000708043A8700080094
:1006B0000708013A870008000708203A8700080069
:1006C0000708103A870008000708083A8700080062
:1006D0003E180516BE1885163E190514BE19851458
:1006E0003E1A8714BE1A07153E1B0714BE1B871639
:1006F000BD1808003F180716BF1887150800B60177
:10070000B301B4013D1C872B3D10BD148A2BC030B2
:10071000BD053D143D083F39B60064008F2B902B7A
:10072000912B922B932B3330B41B8500B41F850182
:10073000B30B8D2BB40B8D2B0310B60CB608031D19
:100740008D2B0030BC003D08BB00DC220800BF1F21
:10075000B22B3F1B07123F1B87153F1F07163F1F7A
:0A0760008711080007128711080036
:084000000200000006000200AE
:02400E00CC01E3
:104200000100030003000300030003000300030098
:10421000030003000300FF00FF00FF00FF00FF009A
:10422000000000000000000000000000000000008E
:10423000000000000000FF00FF00FF00FF00FF0083
:104240000100510005001500550051000500150042
:10425000550051000500FF00FF00FF00FF00FF00B8
:104260000000FF00FF00FF00FF00FF00FF00FF0055
:10427000FF00FF00FF00FF00FF00FF00FF00FF0046
:10428000FF00FF00FF00FF00FF00FF00FF00FF0036
:10429000FF00FF00FF00FF00FF00FF00FF00FF0026
:1042A000FF00FF00FF00FF00FF00FF00FF00FF0016
:1042B000FF00FF00FF00FF00FF00FF00FF00FF0006
:1042C000FF00FF00FF00FF00FF00FF00FF00FF00F6
:1042D000FF00FF00FF00FF00FF00FF00FF00FF00E6
:1042E000FF00FF00FF00FF00FF00FF00FF00FF00D6
:1042F000FF00FF00FF00FF00FF00FF00FF00AA001B
:00000001FF
